:020000040000FA
:0600000020EF0CF01200DD
:02082A000000CC
:04082C006C500CE11F
:100830006896040100513C0BE842E8420D0802E1D1
:100840000ED801D046D808D0040E6C5C03E168963F
:1008500050D802D0000E02D0010E00D01200D9CF25
:10086000E6FFE1CFD9FFE652040104BF046B0301A8
:10087000F86BF06BF16BF66BF76BA6EC07F0DF6AC9
:10088000DF50026E036A010E025C000E03581BE289
:100890000301F15101E017D0F76ADF34FE0BF736A0
:1008A000F66E7F0EF626170EF7220900F5CF02F03E
:1008B0000800F5CF03F004D003C0FAFF0250F96E30
:1008C000FBDFDF2ADDD7EED8E552E552E7CFD9FFCF
:1008D0001200020E0301F05D0AE1A7D8040100BD79
:1008E00003D0C80E006F02D0880E006F01D020D94F
:1008F0001200040E0101FC5D0AE122C46EFF6E507D
:10090000000803E2050EFC6F02D0030EFC6F03012A
:10091000F00512E113D8020E0301F85D04E10401B1
:10092000840E046F08D0040104BD03D0C80E046F08
:1009300002D0880E046F01D0FBD81200D9CFE6FF99
:10094000E1CFD9FF020EE1260301080EF65D000E8D
:10095000F7590EE2F6C3DEFFF7C3DDFFF85103E1FE
:10096000010EF86F04D0F80502E1020EF86F03D013
:10097000080EDE6EDD6A040104930491010EDB5063
:100980000413DFCF05F4000EDB500301F65F010E08
:10099000DB50F75B280EF46F040EF56F0101FDA329
:1009A0001ED0D9CFE9FFDACFEAFFEE50ED1016E006
:1009B000F2C3F6FFF3C3F7FF0800F550F4C3E9FFF5
:1009C000F5C3EAFFEF6E0301F42B000EF523F22BC3
:1009D000F323DF06010E01E2DB06E3D71CD0D9CFFB
:1009E000E9FFDACFEAFFEE50ED1015E0F2C3E9FFC0
:1009F000F3C3EAFFEF50F4C3E9FFF5C3EAFFEF6E7C
:100A00000301F42B000EF523F22BF323DF06010E76
:100A100001E2DB06E4D7020EE15C02E2E16AE552A4
:100A2000E16EE552E7CFD9FF1200D9CFE6FFE1CF63
:100A3000D9FF020EE126030E04010015E76E010E38
:100A4000E7CFDBFF01C4DFFFDE500301F627DD50F7
:100A5000F723280EF26F040EF36FD9CFE9FFDACF38
:100A6000EAFFEE50ED1014E0F2C3E9FFF3C3EAFF32
:100A7000EF50F4C3E9FFF5C3EAFFEF6EF42B000E6D
:100A8000F523F22BF323DF06010E01E2DB06E5D7A7
:100A9000020EE15C02E2E16AE552E16EE552E7CF67
:100AA000D9FF12006D980301F1510CE10401080E09
:100AB000016F200E026F040E036F840E006F04019D
:100AC000046F35D0040120AF22D00301F651040198
:100AD000265D0301F7510401275904E226C4F6F309
:100AE00027C4F7F32BDF0301010EF06F0401080E9A
:100AF000016F200E026F040E036F800E006F040161
:100B0000280E066F040E076FC80E046F10D0030185
:100B1000020EF06F0401056BC80E046F0401080E8D
:100B2000016F280E026F040E036FC80E006F1200D3
:100B3000D9CFE6FFE1CFD9FFE652020E0301F05D07
:100B400036E16D50100B33E004010151026E036A6F
:100B5000080E021801E103502AE100513C0BE84263
:100B6000E8420D0824E10051800B21E1200E026FC4
:100B7000040E036FDF6ADF50026E036A080E025C28
:100B8000000E035813E2DF50EA6A280FE96E040EE4
:100B9000EA22EF50E66EDF50EA6A200FE96E040E9B
:100BA000EA22E552E750EF6EDF2AE5D70DD00301C8
:100BB000F06B0401080E016F200E026F040E036F2C
:100BC0008C0E006F0401046BE552E552E7CFD9FFAC
:020BD000120011
:0E0BD200040120511F0B010801E05BD02051EF
:100BE000600BE842E842E842E842E842010801E0DE
:100BF00051D0245103E0240501E04CD02151230AB7
:100C000048E0010A40E0030A30E0010A25E0240A36
:100C100022E0070A1FE0010A1CE0030A11E0010AB2
:100C200001E038D00301030EF16F0301C80EF26F2B
:100C3000040EF36F0101FD930301080EF66F2AD035
:100C40000301030EF16F0301C80EF46F040EF56F7C
:100C500021D020D01FD01ED00301030EF16F03015D
:100C6000C00EF46F040EF56F15D00301030EF16F83
:100C70000301C00EF26F040EF36F0101FD93030137
:100C8000070EF66F07D00301030EF16F22C4C7F4FD
:100C900001D000D012000401C06BC20EC16F010E62
:100CA000C26FC36BC46BC56B080EC66FB96BB86BF4
:100CB0001A0E726E1E0E736E0401300E166F040E45
:100CC000176F400E146F0401196F380E1A6F040E5F
:100CD0001B6F880E186F0401780E1E6F040E1F6FB5
:100CE000400E1C6F1200D9CFE6FFE1CFD9FF0401FF
:100CF000B86B040118BF30D0FC0EDBCF02F01951E5
:100D0000D880025403E2FC0E19C4DBFF0401B86B67
:100D1000FC0EDB50B85D19E2B851EA6A380FE96E93
:100D2000040EEA22EF50E66EB851E76EFD0EDBCFFF
:100D3000E9FFFE0EDBCFEAFFE750E926000EEA22CC
:100D4000E552E750EF6EB82BE3D70401400E196F60
:100D50001817187D880E18130401B85100D0E552F9
:100D6000E7CFD9FF1200D9CFE6FFE1CFD9FFE65296
:100D70000401B95101E02FD0DF6ADF2ADF50026E93
:100D8000036AFF0E021801E1035001E10BD0FD0ED2
:100D9000DBCFE9FFDB2AFE0EDBCFEAFF01E3DB2A34
:100DA000EF50EBE1DF50026E036AD950FD0FE96EA0
:100DB000FF0EDA20EA6E0250EE5E0350ED5AFD0E91
:100DC000DBCFBAF4FE0EDBCFBBF4DFCFBEF4040101
:100DD000BF6B010EB96FE552E552E7CFD9FF1200A4
:100DE000D9CFE6FFE1CFD9FFE6520401B95101E0C6
:100DF00030D0DF6ADF2ADF50026E036AFF0E02186E
:100E000001E1035001E10CD0FD0EDBCFF6FFDB2A40
:100E1000FE0EDBCFF7FF01E3DB2A0800F550EAE125
:100E2000DF50026E036AD950FD0FE96EFF0EDA2023
:100E3000EA6E0250EE5E0350ED5AFD0EDBCFBAF4BF
:100E4000FE0EDBCFBBF4DFCFBEF40401010EBF6F9B
:100E5000B96FE552E552E7CFD9FF1200D9CFE6FFCF
:100E6000E1CFD9FFE65204011CBF6BD0030E040191
:100E7000B95D01E1B96BB95101E163D0020EB95D11
:100E800006E104011D6B0401030EB96F54D0B905CE
:100E900052E1400E026E036ABE51025C000E03581E
:100EA00003E2400EDF6E02D0BEC4DFFFDFCF1DF4D1
:100EB000DF50BE5DBE6F780EBC6F040EBD6FBF0508
:100EC00015E1DF5012E0BAC4F6FFBBC4F7FF08001B
:100ED000F550BCC4E9FFBDC4EAFFEF6EBC2B000EA9
:100EE000BD23BA2BBB23DF06ECD713D0DF5011E0B4
:100EF000BAC4E9FFBBC4EAFFEF50BCC4E9FFBDC4FC
:100F0000EAFFEF6EBC2B000EBD23BA2BBB23DF061E
:100F1000EDD7BE5110E104011D51026E036A400E6F
:100F2000021801E1035004E10401020EB96F03D07D
:100F30000401030EB96F400E04011C171C7D880EBE
:0C0F40001C13E552E552E7CFD9FF120068
:040F4C00040120512B
:100F5000600BE842E842E842E842E842000901E06A
:100F600055D02151070A51E00B0A4FE0070A40E033
:100F7000010A2CE00B0A28E0020A26E0030A22E01C
:100F8000080A12E0010A0EE00F0A0AE0030A01E073
:100F90003CD00301010EF16F0101040EFC6F36D04D
:100FA00036D834D090D832D00301010EF16F03014E
:100FB000FE0EF26F010EF36F0101FD930301010EAE
:100FC000F66F24D0A8D822D0F4D820D00301010E87
:100FD000F16F040124510301F26FF36BFF0EF2274E
:100FE000010EF3230101FD930301010EF66F0ED0F4
:100FF0000301010EF16F04012451EA6AFF0FE96E4B
:10100000010EEA2222C4EFFF01D000D01200800EB0
:101010000401205D57E12351030A34E0010A10E086
:10102000030A01E04DD00301010EF16F0301B40E7C
:10103000F26F160EF36F120E0301F66FF76B40D0CE
:101040000301010EF16F04012251F66EF76AD89088
:10105000F636F736750EF626170EF7220900F5CF8D
:10106000F2F30A00F5CFF3F3020E0301F76AF2255B
:10107000F66EF351F7220900F5CFF6F30A00F5CF2B
:10108000F7F31ED00301010EF16F04012251F66E39
:10109000F76AD890F636F736790EF626170EF7224D
:1010A0000900F5CFF2F30A00F5CFF3F3F2C3F6FF30
:1010B000F3C3F7FF0800F5500301F66FF76B00D09C
:1010C0000101FD8312000301010EF16F0F0EE66EA8
:1010D000710EE66E0F0EE66E45EC0BF0E552E55232
:1010E000E552010EE66EFF0EE66E010EE66E45EC71
:1010F0000BF0E552E552E55222C4FEF10401225103
:1011000004E10101050EFC6F05D00101060EFC6F24
:101110004BEC06F012000401286B296B04012051EE
:101120001F0B020A14E0030A0EE0010A01E033D0AB
:101130000301010EF16F040128810101FDA102D01C
:101140000401288328D00301010EF16F24D003018C
:10115000010EF16F040124510F0B080DF350036AC7
:10116000000F026E040E03222451800B01E0010ED9
:10117000040DF35003010224F46F000E0320F56FF9
:10118000F4C3E9FFF5C3EAFFEF50040B03E00401E9
:10119000010E286F00D00301F1050AE10301280EBA
:1011A000F26F040EF36F0101FD930301020EF66F5F
:1011B00012000401220510E120511F0B00090CE16F
:1011C0000301010EF16F030E0401215D03E1010132
:1011D000FD8102D00101FD91040122513AE120512B
:1011E0001F0B020836E124510F0B000932E0030106
:1011F000010EF16F040124510F0B080DF350036A27
:10120000000F026E040E03222451800B01E0010E38
:10121000040DF35003010224F46F000E0320F56F58
:10122000030E0401215D07E1840EF4C3E9FFF5C359
:10123000EAFFEF6E0ED024AF06D0F4C3E9FFF5C38A
:10124000EAFFEF6A06D0880EF4C3E9FFF5C3EAFFB0
:04125000EF6E12002B
:0C12540005D91ED902D8FDD71200D9CF51
:10126000E6FFE1CFD9FFE652060E0101FC5D03E384
:101270006D50020B01E0EFD00101F65101E0CFD03B
:10128000020EE66EF20EE66E010EE66E73EC06F0EE
:10129000E552E552E552000952E00101F251640ABB
:1012A0001EE0070A18E0500A12E0010A0CE0030AE7
:1012B00006E0010A01E017D0F46BF56B14D0010EC3
:1012C000F46FF56B10D0F46B010EF56F0CD0010EBE
:1012D000F46FF56F08D0828CF46BF56B04D0829CB0
:1012E000F46BF56B00D0F451E8B08180E8A08190F8
:1012F000F551E8B08186E8A08196F351350A1AE0ED
:10130000010A13E0070A0DE0010A07E0030A01E001
:1013100016D0B90EC06EF96B12D0AA0EC06EF96B62
:101320000ED0AE0EC06EF96B0AD0AE0EC06E5F0E60
:10133000F96F05D0AE0EC06EBE0EF96F00D0010180
:10134000FA6BFB6BF5C1F7F1F451F51168E0F86B3E
:101350000A0EE76EF819E8AE02D0E73402D0E75083
:10136000F85D58E29FD8DF6ADFCF02F0760EE76EB5
:101370000218E8AE02D0E73402D0E750025C47E240
:101380000101F75105E0050EC26E070EC26E04D0D2
:10139000010EC26E030EC26EF45108E0F55106E074
:1013A000F75102E0000E01D0010EF76FF75103E094
:1013B000400EFA2702D0800EFA27DFCF02F0036A30
:1013C00002BE0368F0510224E96EF1510320EA6E77
:1013D000FAC1EFFFDF28026E036A02BE0368F05114
:1013E0000224E96EF1510320EA6EFBC1EFFFF951CF
:1013F00005E0F9C1E6FF2EEC0CF0E552C2B2FED7D3
:10140000C4CFFAF1C3CFFBF1020EDF26ADD7010145
:10141000F82B9ED7010EF66FF46BF56BF86BF605A3
:101420001AE10401B95111E13DD8F0C1BAF4F1C19A
:10143000BBF40401780EBE6F0401BF6B0401010E02
:10144000B96F0101F82B2EEC07F00A0E0101F85DCF
:1014500002E1F86BF66BE552E552E7CFD9FF1200D7
:1014600093969390949C140E6F6E0101FC6B010196
:10147000FD6B0101FE6B0F0E926E3D0EC16E8D0E67
:10148000C06E0101F66BF46BF56BF76B8190819682
:10149000829C12009CEC0AF06FBE02D0BBEC0AF0FA
:1014A0002EEF07F00101F851090A40E0010A39E086
:1014B0000F0A32E0010A2BE0030A24E0010A1DE0D2
:1014C000070A16E0010A0FE0030A08E0010A01E03A
:1014D00032D0000EF06F060EF16F2DD0780EF06F47
:1014E000060EF16F28D0000EF06F050EF16F23D0BD
:1014F000780EF06F050EF16F1ED0000EF06F030E28
:10150000F16F19D0780EF06F030EF16F14D0000E4A
:10151000F06F020EF16F0FD0780EF06F020EF16FC8
:101520000AD0000EF06F010EF16F05D0780EF06F4B
:08153000010EF16F00D0120062
:081538006DA60FD802D06DB6BC
:1015400013D80101FC0508E16DBA06D0686A696A22
:1015500069806988020EFC6F12006D6A696A6D8687
:101560000101010EFC6F12006D6A696A0101FC6BDA
:101570001200B4EF0AF00101FC5101E13AD06850C9
:10158000040B04E06950040B01E03CD86DB231D08B
:101590006850010B04E06950010B01E054D8685019
:1015A000100B04E06950100B01E024D86850400B88
:1015B00004E06950400B01E03BD86850200B04E088
:1015C0006950200B01E036D86850020B04E06950E6
:1015D000020B01E036D8030E0101FC5D01E209D0E7
:1015E0006850080B06E06950080B03E016EC04F0A5
:1015F00068961200698468986D82A19AA08A030097
:10160000A09A12006D926994689412000101FDA1E4
:101610000ED0F8DF6D840201080EFA6F070EFB6F23
:10162000FA07000EFB5BFA51FB11FAE16D94120010
:10163000689C120070A003D098EC05F07090689A36
:101640001200689212006A6A686A9F0E6B6E7B0EC7
:10165000696E6E6A0F0EE66E710EE66E0F0EE66E26
:1016600014D8E552E552E552160E706E68A602D007
:101670006896FCD76D9898EC05F00101FD91010189
:10168000FE6B0101030EFC6F1200D9CFE6FFE1CF24
:10169000D9FFFD0EDBCFE9FFFE0EDBCFEAFFFC0E2C
:1016A000DB5004E0EE6AFC0EDB06F9D7E552E7CF2B
:0416B000D9FF12004C
:0C16B4001201000202000008D8040A0025
:1016C00001000102000109024300020100C03209C9
:1016D000040000010202010005240010010424029C
:1016E0000205240600010524010001070582030804
:1016F000000209040100020A00000007050302407D
:101700000000070583024000000403090434034D70
:10171000006900630072006F006300680069007078
:1017200000200054006500630068006E006F006CCC
:10173000006F0067007900200049006E0063002EF2
:101740000034034300440043002000520053002DA6
:1017500000320033003200200045006D0075006C3F
:10176000006100740069006F006E00200044006595
:10177000006D006F00C616C61609170D174117D267
:011780000B5D
:0E1782002A0EF66E080EF76E000EF86E0201CB
:101790000900F550F56F0900F550F66F03E1F567A4
:1017A00001D03DD00900F550F06F0900F550F16F00
:1017B0000900F550F26F09000900F550E96E0900C3
:1017C000F550EA6E090009000900F550F36F0900B1
:1017D000F550F46F09000900F6CFF7F2F7CFF8F2F1
:1017E000F8CFF9F2F0C2F6FFF1C2F7FFF2C2F8FF4C
:1017F0000201F35302E1F45307E00900F550EE6EE5
:10180000F307F8E2F407F9D7F7C2F6FFF8C2F7FFDB
:10181000F9C2F8FF0201F507000EF65BBFD7120010
:10182000000EF36E00EE00F0040E01D81200EA6024
:1018300002D0EE6AFCD7F350E9601200EE6AFCD7E2
:1018400017EE00F027EE00F0F86A019CC1EC0BF0F7
:0C18500039EC0CF02AEC09F0FBD7120078
:04185C00FF0EE35048
:10186000E84E1200000000D000D000D0E82EFAD7D9
:02187000120064
:02187200120062
:00000001FF
